:108ABB0033302E3520202000003F0006005B004F96
:108ACB000066006D007D0007007F00670077007C6B
:088ADB00009300E50005000016
:10720C0001230001250041068601C100C105C10210
:10721C00C104C101C10342066D000041071E0041BB
:10722C0007700041071A0041071B00012F000124C1
:10723C0000012A0041076C0044068900000000444C
:10724C00070D0000000041067A004407850000008D
:10725C000041076A00410679004107830042071C80
:10726C00000042076E000048078900000000000083
:10727C00000041076102042B7FFFFFFF042600077B
:10728C0086A341076D0041064300480637040007FA
:10729C001D0CA7167E42063F00004206410000422C
:1072AC000644000042064600004506480001020361
:1072BC00004207910000420781000042075F000076
:1072CC0042068700004607623037313635344107B5
:0272DC006B0045
:1057F6004F124B58900907E0FBA3E0FAA3E022F909
:10580600900007124AF8C4540325E02489F582E47F
:105816003407F583E0FEA3E0FF7C047D00124EFD15
:10582600900934124E8E900934E0FCA3E0FDA3E00B
:10583600FEA3E0FFE47BE87A03F9F8124D599009DC
:1058460034124E8E900934E47FFF7EFFFDFCE0F8B3
:10585600A3E0F9A3E0FAA3E022F9900008124AF8BF
:10586600C4135401FFE52FFD3395E0FC74712DF54B
:105876008274073CF583EFF0E92408F9E43AFA026A
:105886004ADF900A0BE0FCA3E0FDA3E0FEA3E0FFE5
:10589600E4F9F8124CCE900A0B124E8E900A0BE0E9
:1058A600FCA3E0FDA3E0FEA3E022AF2FEF3395E0DB
:1058B600FE7C007D0B124B8C746B2FF974043EFA40
:1058C60022AF23EF3395E0FEEF25E0FFEE33FE2215
:1058D6009008FD7B017A0879EAEBF0A3EAF0A3E9E8
:1058E600F022F9900007124AF81313540325E02416
:1058F60089F582E43407F583E0FEA3E0FF227445D0
:105906002FF58274043EF583A3E0C4F8540FC868EB
:10591600FF058222F9900008024AF8900007F91262
:105926004AF8131313540722FF2493F58274063E94
:10593600F583EDF074932FF58274063EF583E0FF50
:1059460090047075F00BEB124ECBEA75F00BA425A4
:1059560083F58322F9900009124AF8C313540322EF
:10596600FDE0FAA3E0FB25E0FFEA33FE74F92FF52C
:105976008274073EF583ECF0A3EDF022900A087CD2
:10598600007D05E0FEA3E0FF024B9EE4FFFEFDFC6A
:10599600D3AB2EAA2DA92CA82B024DF890000512E8
:1059A6004AF8FF900006124AF8FD900004024AF8F1
:1059B600900002F9124C4AFFAEF022F9900007124D
:1059C6004AF8540722900002F9EE8FF0024CA1E04B
:1059D600FF75F00A124ABD90096FF0EF75F00A02E2
:1059E6004ABD900944E0FEA3E0FFC322124CCE8FCD
:1059F600298E288D278C2622FF131313541FFEEFA2
:105A060054C7FFEE045407FE33333354F84F024BAA
:105A160058E0FEA3E0FFE4FCFD22EB5FFFEA5EFE3A
:105A2600E95DFDE85CFC22900944E0FCA3E0FD256D
:105A3600E0FFEC33FE22900A01A3A3E0FEEE22F97A
:105A460090000A124AF8540722AF23EF3395E0FE7E
:105A5600EF7803221582E0C454F04822900A0B1214
:105A66004E8EE47FFF7EFFFDFC22F9F8124CCE90AD
:105A760008C6124E8E9008C622AF2FEF3395E0FE71
:105A860074712FF58274073EF583E05401C43354D4
:105A9600E0FF22F9900006024AF82494F582740683
:105AA6003EF583E022E52E9529F52EE52D9528F580
:105AB6002DE52C9527F52CE52B9526F52B2290091F
:105AC6000AEEF0A3EFF0D3E49FE49E22F9124C1FF6
:105AD600FFAEF022F583E0FCA3E0FDEF25E022F91E
:105AE600900009024AF8900944A3E0FF74017E0081
:105AF600A8070822900944E0FEA3E090047275F01E
:105B06000B124ECBEE22EF9408EE6480948022FFB7
:105B1600ED64015401FE22EF3395E0900944F0A3B1
:105B2600EFF022FFE47BE87A03F9F8024D59900A78
:105B360001A3A3A3E022900003024AF8AF29AE28EE
:105B4600AD27AC2622900679E0FFD36480F8229038
:105B5600097174FFF0900970F090096FF090096E6A
:105B6600F02290092DE0C4F8540FC86822E0FFD354
:105B760064809480900994222401FFE43EFEE43D73
:105B8600FDE43CFC22900686E064012290090AE0CE
:105B9600FEC3EE22248DF974063EFA7401229009A2
:105BA60044124E8E90094422741F2FF58274073ECC
:105BB600F583E0F9A3E0FF22F9900007024AF89086
:105BC6000945E09404900944E064809480223EF5FF
:105BD60083E0F59BE4FFFE2274452FF58274043EB4
:105BE60022900945E025E0FF900944E033FE22902B
:105BF600092CE0C454F04822900644E0FEA3E0FFDE
:105C060022FDE52FFB3395E0FAEBAE0278032290F6
:105C16000A0BA3A3E0FFA3E0900A08CF22E0FFA3AC
:105C2600E0900711CFF0A3EFF022E0FFA3E090078A
:105C360013CFF0A3EFF022E0FFA3E0900715CFF01B
:105C4600A3EFF022900404E0540722FFE4F0A3EF50
:105C5600F022752EFF752DFF752CFF752B7F223ECA
:105C6600F583E01313540322EF3395E0FEEF24EBA4
:105C7600FFEE34FF22900944E0FCA3E0540725E040
:105C8600FF2253A0F743A0102243A00853A0EF22FF
:105C960090096EAFF0EFF0A3E02290096F74FFF069
:105CA60090096E740AF022D3EF64809480227419EE
:105CB6002FF58274082274FFF52EF52DF52C752B21
:105CC6007F22FFEE3395E0FDFC2290092CE0FCA339
:105CD600E02274052FF58274042274252FF5827450
:105CE6000422F9EE8FF0024C82E4900960024E8E97
:105CF600E05438FF900A0522E05407FF900A052277
:105D06001313135401FDEF22F9900001024AF8FD26
:105D1600900005024AF874892FF58274073EF583D0
:105D260022FFEE3AFEED39FDEC38FC22F4FFEEF4EC
:105D3600FE3395E0FDFC22744D2FF58274063EF588
:105D460083225438FFE054C72275BCF990076122BC
:105D56009008D0024E8EFFEEF0A3EFF022FBEDAEE0
:0B5D6600047803227B017A09796E2289
:06503300E4900783F02267
:078E7E009007837401F0224C
:10503C0075FFDE75FFADE4F5E6F5E7C2AF128D71D5
:10504C00900784EFF090068D125C2390068F125C13
:10505C0030900691125C3DE4A3F0A3F0A3F0F5842C
:0E506C00127C1D1287A8128C3912866EE4FF8A
:10507A0075F002EFA42405F582E5F03404F583E027
:10508A00FDA3E0900906CDF0A3EDF0900906125AAF
:10509A00DC24F9F582E4340712597AEF25E02493E7
:0850AA00F582E4340712597A83
:0A50B2000FEFB433C3D2AF128D86A6
:1050BC007F407E0D7D037C00900633125854FBC359
:1050CC00124E0E500F9006331258A5125B7E9006AE
:1050DC0033124E8E12861D900906EFF070030256A5
:0150EC006E55
:1050ED001258B0A374011258E0900906E014B416DA
:1050FD0000400302566E90511175F003A4C583252F
:10510D00F0C583730251530251A70251D50251DBF1
:10511D000251E10252190252C40253EF025401022C
:10512D0054620254820254E00255410255B70255B1
:10513D00D30255F002560B02562E025661025666E8
:10514D0002566B025651E525700302566E1257FA40
:10515D0012595A6403603112587EFFC4135401FD75
:10516D00EF54DF125B15C43354E01257F612591A7F
:10517D00C4135401FFE52FFD3395E0FC74712DF53B
:10518D008274073CF583EFF01257FA12591A542026
:10519D00FF900683E054DF02545EE525700302564E
:1051AD006E1257FA12587FFFC4125D0754BF125B7F
:1051BD0015C4333354C01257F612591A5440FF9088
:1051CD000683E054BF02545E128BB802566E128EE7
:1051DD006E02566EE525700302566E1257FA240ABA
:1051ED001258811259FEEEC39405400D1257FA2440
:1051FD000A12588154C7124B581257FAF990000AE7
:10520D00124AF8900685125D4802545EE52570033A
:10521D0002566E1257FA1259C1600BE92407125843
:06522D008154F80252B1A9
:10523300AF2F1258C974392FF58274083E1258FCE7
:10524300125AC4501AC3E0949990090AE094015089
:105253000E1257FA240712588154F84401804F90D4
:10526300090AE0FEA3E0C39499EE94014013EE947F
:1052730008500E1257FA240712588154F84402803A
:105283002D90090A1259EBEE94084016EF9465EE3F
:10529300940E500E1257FA240712588154F84403FF
:1052A300800C1257FA240712588154F84404124B05
:0152B30058A2
:1052B4001257FA1259C1FF900682E054F802545E64
:1052C400E525700302566E125B8B6003025366126F
:1052D40057FA125921600BE9240712588154C70266
:0252E400535223
:1052E600AF2F1258C974F92FF58274073E1258FC75
:1052F600125AC45017C390090AE09440500E125730
:10530600FA240712588154C744088040125B9294CD
:10531600404013EE9480500E1257FA24071258811B
:1053260054C744108026125B9294804013EE94C0BA
:10533600500E1257FA240712588154C74418800C8D
:0F5346001257FA240712588154C74420124B58AB
:105355001257FA125BBE900682125D484FF0025654
:10536500091257FA12591A5407600812587E54F850
:035375000253D808
:10537800AF2F1258C9125CB43E1258FC125AC450CE
:1053880015C390090AE09440500C1257FA12587F3E
:1053980054F84401803A125B9294404011EE948094
:1053A800500C1257FA12587F54F844028022125BAC
:1053B8009294804011EE94C0500C1257FA12587F04
:1053C80054F84403800A1257FA12587F54F84404D8
:0353D800124B581D
:1053DB001257FA12591A5407FF900683E054F84FEC
:1053EB00F0025609900403E06401F0700302566E5C
:1053FB0012857802566EE525700302566E1257FA27
:10540B002409125881FFC313FEEF54F9FFEE045425
:10541B0003FE25E04F124B58EE6403700A1257FA45
:10542B0012585F4420801A1257FA12595A701512EB
:10543B005A7F12587E54DF1257F6240912588154A2
:10544B00F9124B581257FA125AE55406FF9006847C
:10545B00E054F94F0255ED900686E0FFC374039FAD
:10546B00FFF0BF0105900689800390070D124E9A3D
:10547B00FFFFFFFF02566EE525700302566E125BAF
:10548B008B90090770271257FD12587FFF125D068C
:10549B0054F7125B1533333354F81257F612591A6B
:1054AB005408FF900683E054F74FF080251257FD08
:1054BB0012587FFFC45401FDEF54EF125B15C45417
:1054CB00F01257F612591A5410FF900683E054EF5E
:1054DB004FF0025609E525700302566E125B8B9056
:1054EB00090770291257FD12587FFFC4125D06542D
:1054FB007F125B15C433333354801257F612591A8B
:10550B005480FF900683E0547F4FF080261257FDA6
:10551B002409125881FF5401FDEF54FEFFED640185
:10552B0054011257F6125AE55401FF900684E054C9
:10553B00FE4FF0025609E525700302566E125B8B87
:10554B0070311257FA24091258811259FEEED39476
:10555B0006400D1257FA240912588154C7124B58A2
:10556B001257FA125AE55438FF900684E054C74F8D
:10557B00F080371257FA240A125881FF54F8FEEFC5
:10558B00045407FF4E124B58EFC39407400D1257AC
:10559B00FA240A12588154F8124B581257FA125A1D
:1055AB0045FF900685E054F84FF08052E5257003D7
:1055BB0002566E1257FAF9124ADF64011257F7F9C5
:1055CB00124ADF90067B801AE525700302566E1295
:1055DB0057FA240112588164011257F7125D0E908D
:1055EB00067CF0802E900404E0FF54F8FEEF045488
:1055FB0007FD4EF0EDC394034004E054F8F0801324
:10560B00E525601490067AE004F0C364809483402F
:10561B0002E4F0128A0D804B75250190067A740115
:10562B00F0804020000EE4900402F0128E97C20529
:10563B00C204802FA202B39202300206C20BD20424
:10564B008021C204801D900784E0FF7BFF7A8A795A
:10565B00BB128520800D6325018008127EE080033C
:03566B00127F7D2E
:10566E0030030E900783E07006A3E0FF128D11C287
:10567E00037B017A0879EA128A67EF70030250BC45
:10568E009008ECE0124ED756F20457130556C2148A
:10569E0056B41656BB1756C71A56DB1B56E61D5682
:1056AE00EC1E0000573DD202D20402573DC202C288
:1056BE000402573DD20002573D9008FA1258D912F3
:1056CE004ADFFE900784E0FF6E70648005900784C9
:1056DE00E0FF128D5A02573D128E7E02573D125038
:1056EE003302573D1258D6125B3CFF900784E06F91
:1056FE00703D3002329008FD041258E01259A2FBA0
:10570E0012822080221258D6125B3CFF900784E052
:10571E006F701C3002119008FD041258E01259A24D
:10572E00FB12801712866E900784E0FF128D2A20DE
:10573E00020302567F9008ECE014603814602024B7
:10574E00FB604614607124F9600302567F7B017A78
:10575E000879EA9009031258DF128BD902567F128C
:10576E0057E29008FA1258DF125B3C900402F012D6
:10577E008E97803D1257E29008FA1258DF125B3C6A
:10578E00900402F012866E80281257EC90090012D7
:10579E0058DF125B3CFF1259B0125D15FBC003902F
:1057AE0009001257FD125A9990098AF0D003127D02
:1057BE00A2128E4402567F1257EC9009001258DF47
:1057CE00125B3CFF1259B0125D15FB1270CD128E9A
:0457DE004402567FAC
:1057E200128DBE7B017A0879EA22128DBE7B017A84
:0457F2000879EA2226
:108D710030B60930B7037F41227F422230B7037FEB
:058D810061227F622267
:107C1D009009FEE584F075FFDE75FFAD75840F7577
:057C2D009601758C209A
:107C3200E4A3F0A3F09009FF125A177B407A9CF953
:107C4200F8D3124DF84010900A00E004F070E6906C
:077C520009FFE004F080DEF1
:107C5900E4F58475EF0675840F758A83F597758445
:107C69000F758904F58475B73075840F43890175DB
:107C79008D01758F01758E049009FA124E9A0000D4
:107C89000000E4FF7E01FDFC9009FA125854FBC381
:107C9900124E0E50119009FA1258A5125B7E9009E6
:107CA900FA124E8E80DC438902E58920E41290099C
:107CB900FA124E59E4FB7A01F9F8C3124E0E50E953
:107CC900759702E4F58A9009FEE0F584E4F58412DB
:107CD9008A93128C90128DCF900784E0FF128E1F29
:107CE90043F602128E5A128DDF1288BB9009FA02EE
:027CF9004E8EAD
:108A930075840F75A4CF75A71C75B0E7E4F5E2756F
:108AA300A6FF75E10375E3C0F5A57590FF75ADE30A
:088AB30075AD63F5A5F5842201
:108C9000E4F58443E60875DA3175DB3175DC31754E
:0A8CA000DD3175D983D2DEF58422A0
:108DCF00D2AF759A4075F809759D01C286C2872288
:0A8E5A0075E8C075BCF875D103225D
:108DAC00E4FDFCC3ED9FEC9E50070DBD00010C8053
:018DBC00F2C4
:018DBD002293
:108DDF0075840275E88075BCF975D103E4F58422BA
:1088BB00AB84E4F584F588758DF0F58B758910F52F
:1088CB008E758840900A3A124E9A0000F00DE4F52E
:1088DB008475CC0D75CDF075CA0D75CBF0F5C975DA
:1088EB00C80443A828AF038F84900A3A1258A5FFF7
:0188FB00225A
:108D8600E4F5BB758402900761E0F5BBE4F5844326
:038D9600E71222BF
:108BB800AF231258B27B01900404E04408F09000FF
:108BC8000A125925FF6003BF0406127E43125CBCDB
:018BD800227A
:088E6E00900404E054F7F02227
:107E4300125A9A543FFF7005E5230480071259B074
:107E53007009EF14900A3EF0027ECB125A4FC333DF
:107E6300CE33CED8F9FDAC062493F58274063CF5E7
:107E730083E0D3648094804019125A9A543F14903B
:107E83000A3EF074932DF58274063CF583E014F0FA
:027E9300803637
:107E9500AF231258B27B01900A3F1258DFE5230445
:107EA500900A3EF01259B0900005124B6A125D1609
:107EB500FD125A4FC333CE33CED8F92493F58274CD
:067EC500063EF583EDF01E
:107ECB00900A3EE0C3648094904002E4F0900A3E36
:057EDB00E0FF0289DD5B
:1089DD008523248F239007177401F0A3F0A3F0EFE4
:1089ED003395E0FE90047575F00BEF124ECBEE1241
:1089FD005951E01313135407FFBF0403128E6E2257
:108D9900125C4AFFBF010B90076DE0FF1289DD12DB
:038DA9005CBC228D
:03503900025D71A4
:105D7100C0E0C0F0C083C082C0D075D000C000C0F8
:0D5D810001C002C003C004C005C006C00779
:105D8E00758402C2ED9008C1E5BEF0900761E02473
:105D9E00FD7003025E2C1470030261FE24FD70037D
:105DAE0002621D240560030262799008C1E090082A
:105DBE005D125C517D327F32126E0690076DE0905F
:105DCE000643F090071CE0C4540FFD900469E0C434
:105DDE00F854F0C8A3E0C4540F482D90076DF0D3CB
:105DEE00940F4004E024F0F0900643E0FE90076D1F
:105DFE00E0FFB506046523600D125C4AFEBE020686
:105E0E001289DD125C58900643E0FF90076DE06F3B
:0E5E1E006003128A0D125D4F7403F002627968
:105E2C0090076E125A179008D8124E8E9008DE12F8
:105E3C004E9A000001639008E2124E9A00071C0073
:105E4C00AF231258B27B019008E61258DFE523FD10
:105E5C003395E0FCED125A35125904D582021583A4
:0F5E6C00125A5A9008CCF0A3EFF01259C2602DD1
:105E7B00EDAE047803C333CE33CED8F9125AA0C497
:105E8B005403FF9008E9F01258CA125D1CE0C4F8E5
:0B5E9B0054F0C868FFA3E0C4540F4897
:105EA600800C1258C7125BDEF583E0FFA3E0900872
:105EB600CECFF0A3EFF09008CEE0FCA3E0FDEC130C
:105EC60013543F9008C5F0EC5403FEAF05E4FCFD07
:105ED600A3125A781258A5FFE47B637A01125A700E
:105EE600125854FBC3E49BFF74A89AFE740C99FDE8
:105EF600E498FC9008C6124E8E9008C5E025E02472
:105F060037F582E434061258FC9008C2EEF0A3EF8F
:105F1600F0FBAA06E4F9F89008C61258A5FF124D40
:105F260059125D5690071EE4F09008E61257FD12CE
:105F3600591AC413540720E00302608B12595B649C
:105F4600036003025FCFAF2F1258C9125BDE1258EF
:105F5600FCC39416EE9401500AEF94A4EE9400400C
:105F660002805DC3EF94FFEE9402500AEF94B9EEFF
:105F760094024002804AC3EF94A7EE9406500AEFBB
:105F860094F8EE940540028037C3EF94EBEE940844
:105F9600500AEF9495EE940840028024C3EF9417BC
:105FA600EE940C500AEF94D1EE940B40028011C38C
:105FB600EF945BEE940F500EEF94E9EE940E4006CC
:105FC60090071E7401F002608BE47FC77E01FDFC22
:105FD6009008D0125854FBD3124DF8400C9008D4B8
:105FE600124E9A000002808045E4FF7E01FDFC907F
:105FF60008D0125854FBD3124DF8400C9008D41216
:106006004E9A000001408026E47F8FFEFDFC90083A
:10601600D0125854FBD3124DF89008D44009124EB2
:106026009A000000A08007124E9A000000509008C7
:10603600CCE0131313541F7E00125D5CC3941CEE58
:10604600940050047F0180027F009008CCE0FCA3FE
:10605600E0FDD39404EC940040047E0180027E00AF
:10606600EE5F602C7E00ED54079008CC125D5C64F8
:1060760007600A9008CCE07002A3E0701390071E38
:106086007401F0800B9008D01258A5FFA3124E8E13
:106096007FA37E867D077C009008D4125854FB129D
:1060A60059F27808124E321259F59008E61257FD49
:1060B60012595A601024FD600C24027014125B42BF
:1060C600E47B088006125B42E47B40FAF9F8125939
:1060D600F29008C1E0900859125C517D307F301271
:1060E6006E069008C4E0FF900768E4F0A3EFF09016
:1060F6000465A3E09008C4F0900467E0FFA3E09075
:1061060008DCCFF0A3EFF0E02480F09008DCE03468
:10611600FFF0E0FEA3E0125CC89008D8125854FBCA
:10612600124CCE125D569008D01258A5FF780F1269
:106136004E32125D569008C4E0FFE4FCFDFE900866
:10614600D01258542F125D27A3124E8EE47FFFFE05
:10615600FDFC9008D4125854FBD3124DF8400A9017
:1061660008D4124E9A000000FF9008D41258A5FFDA
:10617600EC33500A9008D4124E9A000000009008A2
:10618600D4A3A3A3E09008C4F0E0FFC41313540300
:10619600A3F0EF543FFFE4FCFDFEA3125A78125819
:1061A600A5FFE47B08FA125A70125854FBC374F820
:1061B6009BFF74039AFEE499FDE498FC125A75124B
:1061C60058A5FF9008C5E0F9F8124E1F9008CAEED0
:1061D600F0A3EFF0125B427808124E321259F5AB7B
:1061E60029AA28A927A8269008CA125A171259F2CE
:0861F600125D4F7404F0807B80
:1061FE009008C1E0FF90085BE4F0A3EFF07D317FE3
:0F620E0031126E0675BCF89007617407F0805C62
:10621D0090063FE0FEA3E0FFA3EEF0A3EFF09008A1
:10622D00C1E0FD90063FE4F0A3EDF0D3EF9480EED6
:10623D009400500EE0948090063FE09400400312CD
:10624D008BB8D3900640E0942590063FE094005023
:10625D0008E50B5404FFEF70089007707401F0808F
:0C626D0005900770E4F0125D4F7402F021
:0C627900900761E0F5BB75840043E8105D
:10628500D007D006D005D004D003D002D001D0006D
:0B629500D0D0D082D083D0F0D0E03217
:0350300002409AA1
:10409A00C0E0C0F0C083C082C0D075D000C000C0EC
:0D40AA0001C002C003C004C005C006C0076D
:1040B700AF231258B290093874011258E0AF24EFB9
:1040C7003395E0FE1258BBA374011258E0125A4F01
:1040D700C333CE33CED8F990093E125B9A1258E01B
:1040E700AF24125A51C333CE33CED8F990094112B7
:1040F7005B9A1258E0C2EDE4FFFEFDFC90078512C3
:104107005854FBD3124DF8401D9007851258A5FF50
:10411700EF24FFFFEE34FFFEED34FFFDEC34FFFC30
:10412700900785124E8EE47F01FEFDFC90078512F5
:104137005854FBC3124DF8700D128D9990078512D4
:104147004E9A00000000AFBFEFFFADBEED90092C07
:10415700CFF0A3EFF0125B4B74809840030242E16B
:0B416700C3EF6480949040030242E12B
:10417200125B1D125B8B707B125CD090094412594A
:1041820066AF03125AF28005C333CE33CED8F9128A
:104192005CC8900689125854125A214D4E4F604BFA
:1041A200125BE774F92FF58274073EF583E0FCA3F6
:1041B200E0FD74932FF582740712597990068912E3
:1041C2005854FBC000C001C002C003125AEC800563
:1041D200C333CE33CED8F9125D32D003D002D00130
:1041E200D000125A20900689124E8E900944A3E004
:1041F20002427A125CD0FD900944E0FAA3E0FB256A
:10420200E0FFEA33FE125CB4125979AF03125AF29C
:104212008005C333CE33CED8F9125CC890070D1295
:104222005854125A214D4E4F6047125BE7125CB44C
:104232003EF583E0FCA3E0FD74B32FF58274071210
:10424200597990070D125854FBC000C001C002C03A
:1042520003125AEC8005C333CE33CED8F9125D3245
:10426200D003D002D001D000125A2090070D124E76
:104272008E900944A3E02410FDFF126E06125AFA32
:10428200125951E01313135407601A125A2D125C7B
:10429200D8125C65125D63C333CE33CED8F9125A9D
:1042A200A054FC4BF0900944E0FEA3E0900473128A
:1042B2005B04125951E0540770030243E4125A2D71
:1042C200125CE0125C65FF25E025E0125D63C333FA
:0C42D200CE33CED8F9125AA054F34BF0B2
:0B42DE000243E4900679E064107038A1
:1042E900125B68FF125BF5FEE4FCFD125BA4125839
:1042F900A5FFE4FB7A04F9F8124CCE125BA412581C
:10430900A5125B29125BA4A3A3E0FFA3E090071CFD
:05431900CFF0A3EFF05E
:10431E000243E4125B4B7411648098500EC3EF6439
:05432E0080949550068B
:03433300EF24EF85
:104336000243CA125B4B74156480985054C3EF64F1
:054346008094A5504C1D
:10434B00125C6EFE125B212420FFE43EA3F0A3EF70
:10435B00F0125CD0900946125966AD03AF05126E90
:10436B0006125AFA125951E05407606D125A2D1267
:10437B005BDE125C66FFC454F0125D63C333CE3355
:0A438B00CED8F9125AA054CF4BF01F
:10439500804D900679E0FDB42510125B68FE125B36
:1043A500F590076EF0A3CEF08035D3ED6480F874F8
:1043B500266480985029900679E0FFC3648094AA0A
:0243C500501D89
:1043C700EF24DAFF900944F0FD125B68FB125BF5FE
:0D43D700FAED1258CA125D1CEAF0A3EBF0DB
:1043E4009009381257FD1259216037900403E07088
:1043F4002290093E1257FD125BBE1258F190093803
:104404001257FD9000091259241249B31257FDF9AD
:10441400EE80281258C7125BAE90093E1257FDC9B0
:1044240080191258C7125CD812590BD58202158311
:10443400125A5AF990093E1257FDC98FF0124C8254
:1044440090093B1257FD125921603A900403E07021
:10445400239009411257FD125BBE1258F190093B9B
:104464001257FDF99000091259251249BD1257FD42
:10447400F9EE802CAF241258C9125BAE9009411298
:1044840057FDC9801BAF241258C9125CD812590BAE
:10449400D582021583125A5AF99009411257FDC95F
:1044A4008FF0124C829009381257FD12591A540792
:1044B4006030900403E0701A90093E1257FD1258C0
:1044C400E89009381257FD125A45FDAB231277EDD7
:1044D40080221258C7743F2FF58274073E1258FC8D
:1044E40080121258C7125CE012590BD58202158350
:1044F400125A5AFE90093E1257FD1259CB90093BAD
:104504001257FD12591A54076032900403E0701ACE
:104514009009411257FD1258E890093B1257FD12B9
:104524005A45FDAB241277ED8026AF241258C97486
:104534003F2FF58274073E1258FC8014AF241258A2
:10454400C9125CE012590BD582021583125A5AFE25
:104554009009411257FD1259CB9009381257FD1298
:1045640059C16034900403E0702190093E1257FD54
:10457400125805FBD3124E0E400A900934124E9A7B
:104584000000FFFF900934A3A380061258C7125DF0
:104594003DE0FEA3E0FF800F1258C7125904D582F4
:1045A400021583125A5AFE90093E1257FD900004D8
:1045B4001259CE90093B1257FD1259C1603690042E
:1045C40003E070219009411257FD125805FBD312E4
:1045D4004E0E400A900934124E9A0000FFFF9009D3
:1045E40034A3A38008AF241258C9125D3DE0FEA392
:1045F400E0FF8011AF241258C9125904D582021564
:1046040083125A5AFE9009411257FDF99000041280
:1046140059CF9009381257FD125921701F90093E45
:104624001257FD125AD29009381257FDF990000919
:104634001259251249B31257FD125CE89009381239
:1046440057FD12591A5407702190093E1257FD1252
:1046540059B69009381257FD125A45FDAB2312770B
:10466400ED90093E1257FD1259CB90071AE4F090D1
:1046740009381257FD12591A131313541F30E02628
:1046840090093E1257FD125AD212870E90071AEF64
:10469400F090093E1257FD125AD212875C90093EDF
:1046A4001257FD125CE890071BE4F090093812578A
:1046B400FD12591AC4540F30E02690093E1257FDDA
:1046C4001259B612870E90071BEFF090093E12574D
:1046D400FD1259B612875C90093E1257FD1259CB50
:1046E4009009381257FD12591AC413131354013088
:1046F400E056900403E0701F9009411257FD125ACE
:10470400D290093B1257FDF990000912592512491C
:10471400BD1257FD125CE890093E1257FD125AD2A1
:10472400E4FCFDC004C005C006C00790094112574F
:10473400FD125AD2125CEFD007D006D005D0041275
:1047440083EF90092EEE801090093E1257FDF91266
:104754004C1FFF90092EE5F0F0A3EFF090093812FA
:1047640057FD125AE530E058900403E07021900997
:10477400411257FD1259B690093B1257FD125A4582
:10478400FDAB241277ED9009411257FD1259CB90DD
:10479400093E1257FD1259B6E4FCFDC004C005C021
:1047A40006C0079009411257FD1259B6125CEFD0AA
:1047B40007D006D005D0041283EF900930EE8013A1
:1047C40090093E1257FDF9900002124C4AFF9009DD
:1047D40030E5F0F0A3EFF09009381257FD12591AA2
:1047E400C41313540390093E30E0351257FD900072
:1047F400041259B9E4FCFDC004C005C006C007900A
:1048040009411257FDF99000041259BA125CEFD015
:1048140007D006D005D0041283EF900932EE801041
:104824001257FDF9900004124C4AFF900932E5F04A
:10483400F0A3EFF090092E125C23900930125C3043
:10484400900932125C3D90076A125B4E7480985056
:094854005DC3EF6480949050559F
:10485D00125B1D125C7BA3EFF0C3EC64809480406F
:10486D000A125BC55005125C8880141259E8940435
:10487D00EE64809480400E125B0C5009125C8F75B3
:10488D00BB000249451259E8125B0D400FEF940C25
:10489D00EE648094805005125C888003125C8F75E5
:0248AD00BB014D
:1048AF0002494590076AE0FFB4100675BB02024942
:1048BF007FEFB41103024961EFB4120302496AEFAB
:1048CF00B41303024973EFB4140302497CD3EF64AA
:1048DF0080F874156480985068C3EF648094A55075
:0148EF006068
:1048F000125C6E125B21125C7BEF04A3F0C3EC64CC
:10490000809480400A125BC55005125C88801412A6
:1049100059E89404EE64809480400D125B0C5008BA
:10492000125C8F75BB00801D1259E8125B0D400FA1
:10493000EF940CEE648094805005125C8880031222
:0E4940005C8F75BB0153A0F8900946E042A0C1
:10494E00802F90076AE0FFB4250575BB038022EF28
:10495E00B4260575BB048019EFB4270575BB058019
:10496E0010EFB4280575BB068007EFB4290375BB9D
:10497E000790076AE0900679F090076A04F0C36426
:0A498E008094AA4002E4F0126ADCF3
:10499800D007D006D005D004D003D002D001D00073
:1049A800D0D0D082D083D0F0D0E032FDAB231277C4
:0F49B800ED90093E22FDAB241277ED90094122CC
:108B2E00EF252FF52FD36480948F4003E4F52FC3E8
:108B3E00E52F648094805003752F0FE52560031296
:038B4E0068E522B5
:1068E500AF0BAE0AAD09AC08124DEB900A01124E82
:1068F5008E1258B0900A0574011258E0125B345498
:1069050001FFEF6016900683E05420FF900A051200
:1069150057FD12587F54DF4F124B58125B34540207
:10692500FFEF6016900683E05440FF900A0512576A
:10693500FD12587F54BF4F124B58125A3C5401FE5A
:10694500EE604A900684E0C31354036403700D900F
:106955000A051257FD12585F44208016900A051249
:1069650057FD12595AFFBF030C125A7F12587E5415
:10697500DF4F124B58900684E05406FF900A05122B
:1069850057FD240912588154F94F124B58125A3C9D
:106995005404FEEE602E900686E0900683B4011145
:1069A500E05408FF900A051257FD12587F54F780EE
:1069B5000FE05410FF900A051257FD12587F54EF4F
:1069C5004F124B58125A3C5408FEEE60339006861F
:1069D500E0B40114900683E05480FF900A05125735
:1069E500FD12587F547F8014900684E05401FF9077
:1069F5000A051257FD240912588154FE4F124B58AF
:106A0500125A3C5410FEEE602D900686E0B4011239
:106A1500900684125CF61257FD240912588154C75A
:106A25008010900685125CFE1257FD240A125881CB
:106A350054F84F124B58125A3C5420FEEE601090F9
:106A4500067BE0FF900A051257FDF9EF124B58122D
:106A55005A3C5440FEEE601390067CE0FF900A0518
:106A65001257FDF9900001EF124B6A125B34544046
:106A7500FFEF602B900686E0B40112900682125C4F
:106A8500F61257FD240712588154C7800E900683CD
:106A9500125CFE1257FD12587F54F84F124B5812D4
:106AA5005B345420FFEF6011900682125CFE125792
:106AB500FD2407125881125A11125B345410FFEF4E
:106AC5006014900685125CF61257FD240A1258814F
:066AD50054C74F124B589C
:016ADB002298
:0576D600900A20EDF018
:1076DB00900646E475F001124BF3FED3E5F0125B16
:1076EB000D401EE4900646F0A3F090064475F001A1
:1076FB00124BF3FEE5F064044E7006900644F0A3C3
:10770B00F0125BFE64034E6006EF64014E70229034
:10771B000646E0FEA3E0FF4E7009900646F0A30478
:10772B00F0800EEF64034E7008900646F0A37407CA
:10773B00F0125BFE2404FD7401A805088002C3331C
:10774B00D8FC900674F0C3900647E0940890064668
:07775B00E0648094805059A6
:107762008F828E83124AF8FF900A22F01258CA744E
:10777200C32FF582748A3EF583E493FC740193FD72
:10778200900646A3E0FB74017E00A803088005C3AF
:1077920033CE33CED8F9FFEC5EFEED5F4E6008903B
:1077A2000674E02BF08005E4900674F0900A22E063
:0777B200C364809480503392
:1077B900802C125BFEEE702BEF14600A146011141A
:1077C900600E2403701D900A21E060028008800E7B
:1077D900900A20E06008900674E02407F022E49003
:0377E9000674F033
:0177EC00227A
:077F7D00E5257003028011ED
:107F84001258B0900A6A74011258E090067AE064BC
:107F9400017028900A6A1257FD125A99543FD394DB
:107FA400004012E92406125881FF54C0FEEF145415
:107FB4003F4E124B58128A0D02800E90067AE064EE
:107FC400027042900A6A1257FDF91259B0FFD36445
:107FD400809481400A90000474FF124B25800BEFBB
:107FE40070089000047413124B6A900A6A1257FDC9
:107FF400F91259B0125C07C333CE33CED8F91259F3
:0D8004002EEFF080057FFF128B2E028A0DFB
:068011007FFF128B2E22FE
:077EE000E5257003027F7726
:107EE7001258B0900A6D74011258E090067AE06457
:107EF700017025900A6D1257FD125A99543FC39489
:107F0700105012E92406125881FF54C0FEEF0454A2
:107F17003F4E124B58027F6A90067AE0640270481F
:107F2700900A6D1257FDF91259B0FFC364809493FC
:107F3700500DEF600A9000047401124B25800BEF7F
:107F4700B41307900004E4124B6A900A6D1257FDB0
:107F5700F91259B0125C07C333CE33CED8F9125990
:107F67002EEFF0128A0D80057F01128B2E028A0DEB
:067F77007F01128B2E2297
:03501200028E2CDF
:0C8E2C00C2CF75840243E8107584003248
:106C7600900686E0B4010790071AE0FC80059007AD
:106C86001BE0FC12595BFF6403601590066FE0FE83
:106C96007401A807088002C333D8FC4E90066FF033
:106CA600900672E0FF124ADFFEEF4E900672F0E0A9
:106CB600FF125D0F25E0FEEF4E900672F012591B93
:106CC600FEC413540730E01390071EE090066F6071
:106CD60006E04410F08004E04420F090066FE0FFE8
:106CE600EEC41313540133333354F8FEEF4EF090D1
:106CF6000686E0900670B4010BE0FF12591BC41320
:106D060013138005E0FF125AE65401FEEF4E90067B
:106D160070F0900686E0FF6401701312591B13137E
:106D260013541F30E021EC9006706017800F125943
:106D36001BC4540F30E010EC9006706006E044026D
:106D4600F08004E04404F0EFB40108125AE613138D
:106D560013800690000A124AF85407FDEDB405099F
:106D6600900671E04420F0803EED7009900671E0D7
:106D76004401F08032EDB40109900671E04402F05E
:106D86008025EDB40209900671E04404F08018ED08
:106D9600B40309900671E04408F0800BEDB40407D3
:106DA600900671E04410F090000A125925FF602108
:106DB600900673E0FE74482FF582E43406F583E00E
:106DC600FF7401A807088002C333D8FC4E900673EF
:016DD600F0CC
:106DD700125BBFFF54076007900673E04410F09002
:106DE7000686E0B4010AEF131313540760108007F7
:0E6DF70012591B54076007900673E04420F009
:016E0500226A
:107A0D00E4900A38F0A3F0900A381259EB9405EE81
:107A1D0064809480501C746F2FF58274063EF5833C
:107A2D00E4F0900A39E004F070DD900A38E004F0DB
:107A3D0080D5E5256004AF2F8002AF231258B29098
:107A4D000A3574011258E0900A351257FDF9126C7F
:107A5D0076125C4AFDBD0109900672E04404F08087
:107A6D000ABD0207900672E04408F0900670E0FF30
:107A7D00900686E033333354F8FEEF4E900670F0E7
:107A8D00300407900672E04410F0900672E0FFE5B6
:107A9D0025C43354E0FEEF4EF0900404E0131313AD
:107AAD00541F90066F30E006E04480F08004E044FF
:107ABD0040F0900673E0FF900403E0C4333354C0EC
:107ACD00FEEF4E900673F0C2FA900A38E4F0A374FC
:107ADD0004F053F87FE59A20E7FB900A38E0FEA307
:107AED00E0246FF5827406125BD40FBF00010EEF18
:107AFD0064324E70F5900A39E024FFF0900A38E0B8
:0E7B0D0034FFF0E0B4FFCBA3E0B4FFC6D2FA21
:017B1B002247
:106ADC00E490096CF0A3F090096C1259EB9403EE5E
:106AEC0064809480501C74742FF58274063EF58378
:106AFC00E4F090096DE004F070DD90096CE004F0B6
:106B0C0080D5E52330E31C900676E0FFE52354079F
:106B1C00FE7401A806088002C333D8FC4F90067699
:106B2C00F08017900675E0FFAE237401A80608806C
:0C6B3C0002C333D8FC4F900675F0C287EE
:106B48001258B090097274011258E0AF2F125A51BE
:106B5800C333CE33CED8F9248DF974063EFA9009A2
:106B68007574011258E09009721257FD125A99541F
:106B78003FFF900978F01259B0900979F0900975A3
:106B88001257FD125A9990097A1259E09009711218
:106B980059E0900970125C99700374FFF0E5256064
:106BA800559009791259D5125C96700374FFF090CC
:106BB8000978E0FFD3648094804007A3E070031253
:106BC8005CA0EF7003125B5590067AE0B4020C12D9
:106BD8005D6A900A217401F0E4801890067AE01248
:106BE8005D6AB40109E4900A21F07D018037E490E0
:106BF8000A21F0FD802F90097A1259D5125C9670FF
:106C08000374FFF0900978E0FF7003125B55125C83
:106C1800AD4009900979E07003125CA0125D6AE446
:086C2800900A21F0FD1276D65E
:106C300090096CE4F0A37402F053F87FE59A20E722
:106C4000FB90096CE0FEA3E02474F5827406125BED
:106C5000D40FBF00010EEF64324E70F590096DE065
:106C600024FFF090096CE034FFF0E0B4FFCBA3E028
:056C7000B4FFC6D2874D
:016C750022FC
:1081A600E4FD7C02900677E4F0A3DCFC7C007D0213
:1081B600E52F30E31C900678E0FFE52F5407FE74A8
:1081C60001A806088002C333D8FC4F900678F080D9
:1081D60017900677E0FFAE2F7401A806088002C349
:1081E60033D8FC4F900677F0C2A57C007D0153F88A
:1081F6007FE59A20E7FB74772DF58274063C125BC7
:10820600D50FBF00010EEF64324E70F5ED1D700103
:098216001CBCFFDABDFFD7D2A5A4
:01821F00223C
:10812800900791E0FFA3E0900781CFF0A3EFF0E57F
:10813800905440FF900791E4F0A3EFF090075FE0C0
:10814800FFA3E0900687CFF0A3EFF0E5905420FF5F
:1081580090075FE4F0A3EFF0900781E07002A3E0DE
:108168007015900791E07002A3E0600B900781E41E
:10817800F0A304F0128E6E900687E07002A3E07000
:108188001C90075FE07002A3E06012900687E4F09D
:0E819800A304F0900785124E9A0000003222D8
:03500C0002667CBD
:10667C00C0E0C0F0C083C082C0D075D000C000C0E4
:0D668C0001C002C003C004C005C006C00765
:10669900C28FAF231258B290099674011258E09034
:1066A900076CE0FF2462F582E43407F583E0900982
:1066B90093F0EF14603E1460651460741470030263
:1066C900675F14700302678D240560030267A89051
:1066D9000711125A17900999124E8E90099912585A
:1066E9004DFBD3124E0E402F900999124E9A00007D
:1066F900FFFF8023900713125A17900999125A65C0
:10670900900999125854FBD3124E0E400A900999D8
:10671900124E9A0000FFFF900999A3A380039007E6
:1067290015E0FFA3E0900994CFF0A3EFF00267A86A
:106739009009961257FDF9124ADF603F9007181227
:106749005B73400474FF8001E4F0A3F0125CAD4078
:106759004E90071880469009961257FD125D0E60FB
:106769001A900719125B73400474FF8001E4F0A3C7
:10677900F0125CAD40299007198021900994E4F04A
:10678900A3F0801B900717125B73400474FF80010C
:10679900E4F0A3F0125CAD4006900717E014F0C2D4
:1067A9008653F87FE59A20E7FB900993E0F59BE48F
:1067B900FD0DEDB432FB900994E0FF7E0053F87FA4
:1067C900E59A20E7FB8F9B7D000DEDB432FB900924
:1067D90094A3E0FF7E0053F87FE59A20E7FB8F9BA7
:1067E9007D000DEDB432FBD28690076CE004F0C356
:1067F90094064002E4F012812890076BE024FA60C5
:106809000924067008127A0D80031281A690076B7D
:10681900E004F0E05407F0125C4A60076401600389
:106829000268AB125B42C31259974006125AAB0277
:0F68390068C412599140030268B8125991507CFB
:1068480090099DE4F09009961257FDF990000A12FC
:10685800592524FE601014601C2402702B12595B09
:1068680064036024801C900770E0701C12595B64FC
:10687800036015800D900770E0600D12595B64038A
:10688800600690099D7401F090099DE0602E9004C7
:1068980004E0FF131313541F30E021127E43125CEF
:0168A8005897
:1068A90080191259914003125AAB125991500C7523
:1068B9002E00752D00752C00752B00758DF0758BCC
:0168C90000CE
:1068CA00D007D006D005D004D003D002D001D00022
:0B68DA00D0D0D082D083D0F0D0E032CC
:0683EF0090095C124E8EA5
:1083F500AF2EAE2DAD2CAC2B780F124E32900964FA
:10840500124E8E900964125854FBC3E49BFFE49A04
:10841500FE740199FDE498FCA3124E8E90095C123E
:1084250058A5FF900968125854FB124CCEC004C0E1
:1084350005C006C0079009601258A5FFA31258543D
:10844500FB124CCED003D002D001D000EF2B125D31
:06845500277810124E1FF3
:01845B0022FE
:10875C007C027D8F124B9E7C027D8F124B8C7C0495
:10876C007D00124EFD900A42124E8E900A42125813
:10877C00A5125B29900A42125A65900A421258546B
:10878C00FBD3124E0E400A900A42124E9A0000FF82
:0B879C00FF900A42A3A3E0FEA3E0FF51
:0187A70022AF
:10870E00900A73EEF0A3EFF0C374469F74019E506F
:10871E003A900A73125A177BAA7AFEF9F8124DF89C
:10872E004029900A737C027D8F125989900A73EC4E
:10873E00F0A3EDF0C3943CEC9400400CD3E09458BD
:0E874E00900A73E0940240037F01227F002214
:0B77ED00900A08EEF0A3EFF0A3EDF00F
:1077F80014601E14602B14603814604524FE605118
:10780800240660030278B6125982900A08EE0278BC
:10781800B2125982EF2430FFEE3433900A0802780E
:10782800B2125982EF2460FFEE3466900A0802789B
:10783800B2125982EF2490FFEE3499900A08027828
:10784800B2125982EF24C0FFEE34CC900A080278B5
:10785800B2AF03E4FCFDFE900A0B124E8E7BFF7A5A
:10786800FF125888FF7804124E1F900A0B124E8E92
:107878007B297A04125888FFE4FB7A04F9F8124D40
:107888005912589C2400FFEE3408125B83125A6286
:10789800900A0B125854FBD3124E0E400A900A0B52
:1078A800124E9A0000FFFF125C15F0A3EFF0900A49
:1078B8000AE064066036900A08E0FEA3E0FF7C0454
:1078C8007D00124EFD12589C125B29125A62900AD2
:1078D8000B125854FBD3124E0E400A900A0B124E4C
:1078E8009A0000FFFF125C15F0A3EFF0900A08E081
:0478F800FEA3E0FF0C
:0178FC002269
:10857800E4FFEF75F008A4248DF582E43406125A5E
:10858800DA241FF582E4340712597AEF75F008A44B
:10859800248FF582E43406125ADA243FF582E43453
:1085A8000712597AEF75F008A42491F582E434068D
:1085B800125ADA244DF582E4340612597A0FEFB4D0
:0285C80010B0F1
:0185CA00228E
:1072DE004208BF000042086A00004208650000C173
:0572EE0008C107C10604
:1086BF00900865E475F001124BF3FCE5F064404C53
:1086CF0022D39008C0E094009008BFE064809480AB
:1086DF0022E0FEA3E0246CF582740822E0FBA3E005
:1086EF00FAA3E0F98E8275830022900865F0A3F05B
:0F86FF0022900861E004F022900860E004F0226D
:0A8E6400C207C208E4900869F0227A
:108BFA00E49008BFF0A3F090086AF0A3F0A3F01283
:108C0A0086F9900860F0A37440F0E4900868F022B6
:068E8500128E64028BFA5C
:108CF800E4F5848FC343C30175C04475CF8EC2C3E6
:098D080043E60290086704F02222
:108DBE00E4F58420C7FDC2C2128E85E4900867F0E8
:018DCE002282
:0B8E4400E4F584D2C290086704F0221D
:0D8E1F00AE07128CF8900864EFF0028E850B
:108B0900E4900A75F0A3F0300702FF222008FDD295
:108B190007900862E4F0A37410F09008ADEFF0E458
:048B2900A3F07F0135
:018B2D002225
:1089A90030070A900862E07002A3E070037F00229A
:1089B900900863E024FFF0900862E034FFF090082B
:1089C900AEE0FE04F074AF2EF582E43408F583EFCF
:0489D900F07F012208
:0B8E4F00300707C207D2081250212292
:0E502100AF84E4F58420C7FDC2C4D2C58F84DD
:01502F00225E
:10838000900A10EBF0A3EAF0A3E9F0900867E07020
:1083900002FF22900A13E0FE6005D3941040037F91
:0883A0000022128B09EF60447A
:1083A800E4900A15F0900A13E0FF900A15E0FEC366
:1083B8009F501A900A101286EB124AF8FF1289A9E8
:1083C800EF7002FF22900A15E004F080D8E49008CC
:1083D80069F0128E4F900A14E070032008FD90088F
:0483E80069E0FF2227
:0383EC007FFF22EE
:0E7CFB00900A46EBF0A3EAF0A3E9F0A3EDF047
:107D0900E4FF1286D050012253E6FD9008651286E1
:107D1900E03EF583E0FF1286BF70031286F91287F1
:107D2900007003128707E4FE900A49E0FDEEC39D47
:107D3900502FEEC39F502A900865E0FC1286E23C62
:107D4900F583E0FD900A461286EBED124B6A128626
:107D5900BF70031286F912870070031287070E801D
:107D6900C7EEC39F50131286BF70031286F912879C
:107D79000070031287070E80E89008C0E024FFF026
:107D89009008BFE034FFF043E602900A49E0FEEFB5
:087D9900C39E50028002AF06F8
:017DA10022BF
:0C8E38001286D040047F0180027F0022DF
:03501800026F76AE
:106F7600C0E0C0F0C083C082C0D075D000C000C0E1
:036F860006C0073B
:106F8900C20DAFC1EF124ED76FBF086FBF106FCFE1
:106F9900186FD4206FE128700E3070193870216095
:106FA900701C68702170701C78702980702990702D
:106FB90099A0000070A79008ADE0F5C2C2C590087D
:106FC900ACE4F00270A99008AE802890086974FDBD
:106FD900F0D2C4D2C50270A99008AEE0FF9008AC07
:106FE900E0C39F5014E0FF04F074AF2FF582E4343E
:106FF90008F583E0F5C20270A9D2C4900869E4F0EB
:10700900C2080270A9D2C590086974FEF00270A97D
:1070190002709ED2060270A990085FE4F00270A97E
:1070290090085FE07020E5C2F0E0FFC3900861E0DE
:107039009F7480F8900860E06480985003128BFA7E
:1070490090085FE004F0900861E024FFF090086088
:10705900E034FFF090086A1286E03EF583E5C2F05D
:1070690090086AE475F001124BF3FEE5F064404EB6
:10707900700690086AF0A3F090085FE014F07020A1
:107089009008C0E004F070189008BFE004F0801088
:1070990030060DC2069008ACE4F0D2C58002D20DCC
:1070A900300D0EC2C6D2C6C2C5C2C4D2C2C20DC23A
:0370B90008C2C347
:1070BC00D007D006D000D0D0D082D083D0F0D0E092
:0170CC003291
:058E8B00A2C7E433FF63
:018E900022BF
:1085CB00EFF0A3ECF0A3EDF0A3EBF0A3EAF0A3E93B
:1085DB00F0227403F0A374E8F0A3E584F0E4F584CF
:1085EB0022D2C4D2C5D2C2C2C3E4900A7CF0FF220D
:1085FB00E0FBA3E475F001124C09A9F0FA22E02587
:10860B00E044A0F5C27F032274FFF5F0124BF34553
:02861B00F0224B
:068E9100C2C253E6FD22FF
:0678FD0090097B1285CB0F
:107903009009841285DD20C7FDC2C4D2C2D2C5E46A
:10791300FF900A7CF030C3FDAEC1EE24F86023244F
:10792300F8601F24F8602924F8603024F8603424B8
:10793300F870030279C024F870030279C82438026E
:1079430079D0EF700690097B128609C2C50279D6F9
:1079530090097CE0F5C27F050279D6900A7C740316
:10796300F08070EFB4050B90097CA3E0F5C27F06AD
:107973008061EF64067034900983E090097E70059E
:107983001285FB8008E0FBA3E0FAA3E0F9124ADFCB
:10799300F5C2900982E024FFF0900981E034FFF002
:1079A300E07002A3E0702C7F078028EFB40706D2B3
:1079B300C47F09801E900A7C7405F08016900A7CAF
:1079C3007404F0800E900A7C7406F08006900A7CA2
:1079D3007401F0EFB40904C2C38025900A7CE0B4BB
:1079E300030B90098412861360031285EC900A7CC2
:1079F300E06008C2C5D2C4C2C38005C2C3027918FD
:097A030020C7FD900986E0F5841E
:017A0C002257
:0675AC0090099E1285CB40
:1075B2009009A61285DD20C7FDD2C2C2C4D2C5E49D
:1075C200FF900A7CF030C3FDAEC1EE124ED775F5C6
:1075D2000075F80875F810761D1876282076302880
:1075E200764B30765338765B40766B507693580004
:1075F2000075F5027699C2C5EF700990099E128650
:107602000902769FEF6401600302769F90099EE073
:1076120025E044A1F5C27F0402769F90099FE0F520
:10762200C27F0502769F900A7C7403F0806FEFB4EC
:10763200050B90099FA3E0F5C27F068060EFB406B8
:1076420006D2C57F0180568018900A7C7404F080AF
:107652004C900A7C7406F08044EFB404047F0280EC
:107662003C900A7C7405F080349009A11285FBE5F8
:10767200C2124B589009A5E024FFF09009A4E0340F
:10768200FFF0E07002A3E07004C2C280107F0280AB
:107692000CD2C47F098006900A7C7401F0EFB40911
:1076A20004C2C38025900A7CE0B4030B9009A612A1
:1076B200861360031285EC900A7CE06008C2C5D292
:1076C200C4C2C38005C2C30275C720C7FD9009A802
:0376D200E0F5845C
:0176D5002292
:107348009009C8EFF09009CB1285D49009C9ECF0E8
:03735800A3EDF0B2
:10735B00753200543FF533543F6058C37440953336
:10736B00FFE49532FE9009CEE0FCA3E0FDC39FEC59
:10737B009E50068C308D3180048E308F3112744CC0
:10738B0060037F02229009CAE02531F09009C9E021
:10739B003530F09009D0E0700B9009CCE530853199
:1073AB00F0124BF3C39009CFE09531F09009CEE08A
:1073BB009530F09009CEE0F530A3E0F531D3E5310F
:1073CB009400E53094004076E5319440E53094002C
:1073DB00500F12744C60037F0222E4F530F53180BC
:1073EB00DC9009C8E0FFA3E0FCA3E0FDA3E0FBA356
:1073FB00E0FAA3E0F9900981E4F0A37440F090095E
:10740B00D0E0900983F01278FD900A7CE060037F56
:10741B00022274C02531F53174FF3530F5309009F7
:10742B00CAE02440F09009C9E03400F09009D0E0A4
:10743B00708B9009CC75F040124BF30273C87F0030
:10744B00229009C8E0FFA3E0FCA3E0FDA3E0FBA3AF
:10745B00E0FAA3E0F9900981E530F0A3E531F09073
:0F746B0009D0E0900983F01278FD900A7CE022AE
:108D43009009A4E4F0A304F01275AC900A7CE060EF
:078D5300037F01227F0022D3
:108CAA00900A7BEBF07B017A0A797B9009CEE4F09B
:0A8CBA00A304F0E4A3F012734822B3
:108B7400C0079009E0E0FFA3E09009A4CFF0A3EFC1
:108B8400F0D0071275AC900A7CE060037F01227F6D
:028B94000022BD
:108CC400C0079009E8E0FFA3E09009CECFF0A3EF3E
:0A8CD400F0E4A3F0D0071273482269
:108CDE007B01E4900A27F0227422F0A3EFF0A32286
:0A8CEE007B01E4900A27F07D0422C8
:0E87F000900A23EBF0A3EAF0A3E9F0A3EDF06A
:1087FE00E4900A28F0900A23E0FBA3E0FAA3E0F944
:10880E00A3E0900A13F0900A27E0900A14F0E4FF18
:10881E00128380EFB4FF0D900A28E0FE04F0EEC341
:06882E00940340D17E001E
:018834002221
:0B8A6700900A70EBF0A3EAF0A3E9F026
:108A72007E007F007D10124F2A900A70E0FBA3E077
:108A8200FAA3E0F97D10127CFBEF7002FF227F0156
:018A920022C1
:108520009009B4128CE67413F0124ADF9009B7F088
:10853000900001124AF89009B8F0900002124AF82F
:108540009009B9F0900003124AF89009BAF090002F
:1085500004124AF89009BBF0900005124AF89009FD
:10856000BCF0900006124AF89009BDF07A0979B47F
:08857000128CDE7D0A0287F087
:108D1100900A4A128CE67403F0A374FFF07A0A7980
:098D21004A128CDE7D040287F089
:108D5A00900A4E128CE6741CF0A374FFF07A0A791A
:078D6A004E128CEE0287F0AF
:108D2A00E4900A52F0A3EFF0A3740AF0A3EFF07AEA
:098D3A000A7952128CEE0287F056
:108C1A00E0FEA3E0A60608F6E4F584C2AF43B70176
:0F8C2A0022E475F001024C09EEF0A3EFF0A32253
:10897200AB84A2AF920EE4FCFDED900A56124E8E2D
:10898200900A58781E128C1A438F02438F0118E600
:10899200FE08E6F5828E83E4F053B7FEF58FA20E51
:0689A20092AFAF038F84C9
:0189A80022AC
:02887900AB054D
:10887B00AA84A2AF920FE4FCFDED900A5A124E8E21
:10888B00EBFF3395E0FEEFF44E601C900A5C7834FE
:10889B00128C1A758F0118E6FC08E6F5828C83EBB7
:0F88AB00F053B7FEE4F58FA20F92AFAF028F84A8
:0188BA00229B
:1084C200900A29128C32ECF0A3EDF0A3EAF0A3EBB0
:1084D200F0900A2DE07002A3E06042900A29E0FECB
:1084E200A3E0FFA3E0FCA3E0F5828C83E0FD128809
:1084F20079900A2EE024FFF0900A2DE034FFF090EC
:108502000A2CE004F07006900A2BE004F0900A2A8C
:0E851200E004F070BC900A29E004F080B4226E
:088E7600E4900000F0A3F022DB
:108AE300900000E0FEA3E0FF128972900000E0FE18
:108AF300A3E0FF7C007D027B007A041284C2E49031
:068B03000000F0A3F022C7
:0A80A700A905900A2FEEF0A3EFF0F8
:1080B100EE54FCFE900000E0FCA3E0FD7002EE6CCB
:1080C100604CED4C6003128AE3900A2FE0FEEE54FF
:1080D100FCFE7F00900000F0A3EFF0900A31128CBB
:1080E100327400F0A37402F07E04900A31128C2BDA
:1080F10085F082F583E493FD900A33128C2B85F091
:1081010082F583EDF0EF1F70011EEF4E70DC900AD7
:108111002FE0FCA3E0FDEC5403FC74022DF5827406
:06812100003CF583E9F0CB
:018127002235
:1088FC00900A16128C32EBF0A3EAF0A3E9F0900A7E
:10890C001B74FFF5F0124C0945F0601E900A16120C
:10891C008C2BAFF0FE900A18E0FBA3128C2BA9F065
:0B892C00FA124ADFFD1280A780D4225F
:10829800E47F01FEFDFCE0F8A3E0F9A3E0FAA3E027
:1082A800FB22128835900950124E8E900949E0251C
:1082B800E024F9F582E43407F583E0FEA3E022FB2D
:1082C800C374FF9BFF740F9EFEE49400FDE49400CA
:1082D800FC22900948E075F002A42405F582E5F037
:1082E800340422900949E025E02493F582E4340718
:1082F80022E47BFF7A0FF9F822E0FCA3E0FDA3E07B
:05830800FEA3E0FF22CE
:086E0600900948EFF0A3EDF044
:106E0E001282EF1282C0FBAA061282B3FFC3EF9B5F
:106E1E00FFEE9A1282D090094C124E8EE490094ADF
:106E2E00F0A3F07F0FFEFDFCA312829EC3124DF85D
:106E3E00400890094AE4F0A304F074FF7FF1FEFDD0
:106E4E00FC90094C12829ED3124DF8500874FF909C
:106E5E00094AF0A3F090094AE0FEA3E0FF4E70034A
:0B6E6E00026F75EFF47002EEF470612B
:106E79001282EB1282C0FFE4FCFD900958124E8E7B
:106E8900900958128298C3124DF8500A9009581265
:106E99004E9A000000011282DA1282C0FFE4FCFD62
:106EA9001282FA124CCE90095812829E1282AAFFBF
:106EB900E4FCFD90095012829E124CCE90095412A6
:0E6EC9004E8E1282F990095412830112883500
:0F6ED700026F4890094AE07004A3E06401706FF5
:106EE6001282DA1282C01282C71282F9124CCE9036
:106EF6000950124E8E1282EB1282C01282C790097E
:106F060054124E8E900954128298C3124DF8500AAC
:106F1600900954124E9A0000000190095012830104
:106F2600A312829E1282AA1282C790095012829ED2
:106F3600124CCE1282F9128835C374FF9FFF740F6C
:0F6F46009EFE1282DAF583EEF0A3EFF0128A0DB1
:106F5500900949E0FF25E024F9F582E43407F5833B
:106F6500E0FCA3E0FDEF1282EFF583ECF0A3EDF07A
:016F750022F9
:108DEF000001FF00FF000001010000FF00FF010074
:1072F300040800000000041A000000000416000047
:10730300000002130000011500010D00020E000031
:1073130003100000004409140000000044090C009D
:107323000000004209120000410910004109110048
:10845C00AF0BAE0AAD09AC08024DEB900914E0FC71
:10846C00A3E0FDA3E0FEA3E0FFEC4D4E4F229009EC
:10847C00EAA3A3E0FEA3EE229009EAA3A3A3E022C1
:10848C00FFE4FEFDFCEF22AFB0FEEF5407FFE478F3
:10849C0010024E46EF4BFFEE4AFEED49FDEC482232
:1084AC00900A5FE0FBA3E0FAA3E0F9229009EAA3AB
:0684BC00E0FDA3A3ED2288
:1087A800D2B3C2B4128B96E4FCFDC004C005C00667
:1087B800C007128493D003D002D001D0001284A045
:1087C8008F198E188D17F5168F1D8E1C8D1BF51A97
:1087D800AF907513008F147B017A0979188B108A72
:0887E8001189128A0E890F228B
:05830D00900A5EEFF094
:10831200E50F2401FFE4350EFAA907A37401F0A3C7
:10832200EAF0A3E9F01284AC740190092C6B700896
:10833200E965827003EA6583700D900A5F04F0A319
:108342007409F0A37418F01284ACE51085118385CA
:1083520012826B7008E965827003EA6583601E9081
:108362000A5EE0850F82850E83F0900A5FA3E0FA31
:0D837200A3E0AE028E0EF50F900A5EE0F063
:01837F0022DB
:10861D0053E6F7E5108511838512826401700AE532
:10862D000F65827004E50E65837003FF802FAB101C
:10863D000512E512AA117002051114F9124ADFFF95
:10864D00740190092C6B700AE51265827004E511B6
:10865D006583700975100175110975121843E608C7
:01866D0022EA
:03501E000262A08B
:1062A000C0E0C0F0C083C082C0D075D000C000C0C4
:1062B00001C002C003C004C005C006C00720DF0340
:0362C0000265F084
:1062C300E50C6005D50C02D210128B96E4FCFDC0E0
:1062D30004C005C006C007128493D003D002D001C6
:1062E300D0001284A08F0B8E0A8D09F508AF1DAE66
:1062F3001CAD1BAC1AAB0BAA0AA909F8C3124E0EAC
:106303006031E50B651DFFE50A651CFEE509651BAC
:10631300FDE508651AFC9009EA124E8E9009EA120F
:10632300846A6003751503850B1D850A1C85091B8B
:1063330085081AE51570030265441515E515600314
:10634300026544E519650BFFE518650AFEE5176567
:1063530009FDE5166508FC9009EA124E8E12848445
:106363005401FFEF601012845CEF540112848C60BF
:10637300057F0112830D1284845402FFEF60101213
:10638300845CEF540212848C60057F0212830D1229
:1063930084845404FFEF601012845CEF540412846D
:1063A3008C60057F0312830D1284845408FFEF6011
:1063B3001012845CEF540812848C60057F041283EE
:1063C3000D1284845410FFEF601012845CEF54109C
:1063D30012848C60057F0512830D1284845420FF80
:1063E300EF601012845CEF542012848C60057F06EA
:1063F30012830D1284845440FFEF601012845CEF0B
:10640300544012848C60057F0712830D12848454D8
:1064130080FFEF601012845CEF548012848C60055F
:106423007F0812830D12847A5401FEEE60121284E7
:106433005CEE5401FEE4FDFCEE60057F0912830D62
:1064430012847A5402FEEE601212845CEE5402FE51
:10645300E4FDFCEE60057F0A12830D12847A540476
:10646300FEEE601212845CEE5404FEE4FDFCEE606A
:10647300057F0B12830D12847A5408FEEE6012120C
:10648300845CEE5408FEE4FDFCEE60057F0C128391
:106493000D12847A5410FEEE601212845CEE5410D6
:1064A300FEE4FDFCEE60057F0D12830D12847A5429
:1064B30020FEEE601212845CEE5420FEE4FDFCEE3E
:1064C30060057F0E12830D12847A5440FEEE601233
:1064D30012845CEE5440FEE4FDFCEE60057F0F1277
:1064E300830D12847A5480FEEE601212845CEE54A3
:1064F30080FEE4FDFCEE60057F1012830D1284B86C
:106503005401FDED601312845CE4FEED5401FDE4DF
:10651300FCED60057F1112830D1284B85404FDED68
:10652300601312845CE4FEED5404FDE4FCED6005AD
:106533007F1312830D850B19850A188509178508A2
:1065430016C2DF12845C9009EE124E8E900914E09D
:10655300FCA3E0FDA3E0FEA3E0FF90090C124E8E26
:106563009009EEA3E0FDE4FFFEED5402FDE4FC9090
:106573000914124E8E128467604090090C12846ACB
:106583007006900912F0A3F0900913E004F070066E
:10659300900912E004F0D3900913E0945890091283
:1065A300E0648094824046900911E070057F1612E2
:1065B300830D9009117401F08033128467702E905B
:1065C300090C12846A6026900912E0FEA3E0FFD34F
:1065D300940AEE64809480400FEF9458EE648094A4
:0D65E3008250057F1212830D900911E4F023
:0A65F000900910E004F064027067E7
:1065FA00E59054039009EAF0E0FDFFE5146F5403B7
:10660A006050E514AE137802C333CE33CED8F97E88
:10661A0000540CFFED5403FDEF4D24EFF582EE34E8
:10662A008DF583E493FF9009EBF0A3E50DF0EF25D8
:10663A000DF50DE0650D30E1109009EBE0B40104B1
:10664A007F1480027F1512830D9009EAE07513000A
:07665A00F514900910E4F0B3
:10666100D007D006D005D004D003D002D001D0008D
:0B667100D0D0D082D083D0F0D0E03237
:108B9600D2B4E4FBC2B3ED25E0FDEC33FC30B50402
:108BA600ED4401FDD2B30BEBB410E9C2B4AF05AE90
:018BB60004BA
:018BB700229B
:107333004109F200C10AC1094709F318100C0806F4
:02734300040341
:108B5100900474E0C3135403FF2290000A124AF8F0
:108B61001313135407FF22900A62E0FBA3E0FAA358
:038B7100E0F92206
:108BD900900003124AF82406600D14601014600A0C
:108BE9002404700C02747A028C58028DFF128E0FC5
:018BF9002259
:108C5800D20AE49009F2F0128B51BF030E9004047B
:0C8C6800E04408F0E4FF1289DDD209228C
:108DFF00C20A128B51BF0307900404E054F7F0220C
:108E0F00D20A128B51BF0307900404E04408F022EA
:10747A00AF23EF3395E0FE7C007D0B124B8C746BCF
:10748A002FF974043EFA900A627401F0A3EAF0A399
:10749A00E9F0200A030275AB9009F2E0FF04F0EF6D
:1074AA00B460037401F0128B68900009124AF8C3A1
:0A74BA00135403640360030275AB72
:1074C400AF23EF3395E0FEEF25E0FFEE33FE744586
:1074D4002FF58274043EF583E0FEA3E0FFD3945BB2
:1074E400EE940F4007E4900A65F08058D3EF9417A8
:1074F400EE940C4008900A657401F08047D3EF9431
:10750400EBEE94084008900A657402F08036D3EFDD
:1075140094A7EE94064008900A657403F08025D37E
:10752400EF94FFEE94024008900A657404F080140E
:10753400D3EF9416EE9401900A6540057405F0802B
:10754400037406F09009F2E024FFFFE434FFFE9098
:107554000A65E024F3F582E43409F583E0FD33950C
:10756400E0FC124B9EED703F300903C209229004E7
:1075740004E0131313541F30E02D128B68128B5B3D
:1075840064016015BF0206900770E0600C128B5B0B
:10759400BF0314900770E0600E127E4374FFF52E53
:0775A400F52DF52C752B7F7E
:0175AB0022BD
:02734500C10B7A
:104F56009009B0E0FF75F018A42402F582E5F0345C
:104F6600A4F583EF2583AF8222124B58900A67E09F
:104F7600FBA3E0FAA3E022FE7A0479037B01900A00
:104F86001B7401F0A37418F022AFF0FEE0FCA3E05E
:104F9600F5828C83E493FD229009ACF0A3EFF0E454
:104FA6009009B2F0A3F02275F018EEA42402F5825F
:104FB600E5F034A4F583EE2583AF8222F9E43AFACC
:104FC600024ADF7E007C017D18124B8C74022FF999
:104FD60074A43EFA22EFF0A3EDF0A3EBF0A2AFE447
:104FE60033A3F0C2AF22E475F001024C099009B375
:104FF600E004F0229009B2E004F022FDEDFFEEF0AD
:05500600A3EFF0E4221D
:108A0D00300027200B263002237F407E0D7D037C16
:108A1D0000900633E0F8A3E0F9A3E0FAA3E0FBC36E
:0D8A2D00124E0E7002D203D20B22D2042290
:058A3A00900A77EFF047
:108A3F00128E76E4900A78F0900A77E0FFA3E0FEBA
:108A4F00C39F5011124FAD124F7D1288FC900A78C0
:088A5F00E004F080E3028AE369
:10893700900A797402F0E4A3F0128E767EA47F0089
:108947007A0A79791289647EC47FD27A0A797A128F
:0D8957008964128AE3127B1C7F1E028A3A9B
:0E8964007B01900A1BE4F0A304F01288FC22B1
:108C3900E5B030E01190C4D2E493F4600990A40047
:0F8C4900E49364026003128937E4900402F0227E
:10866E00C20B900402E0FFC3941E503A124FC97B16
:10867E00FF78037C047D017E017F18124A97E4FF88
:10868E0075F00BEFA42473F582E5F03404F583E066
:10869E00C4135401FE74712FF582E43407F583EE92
:1086AE00F00FEFB410DA900633124E9A000000006D
:0186BE002299
:108C7400900402E0C3941E5012128E7690040212E5
:0C8C84004F59124F7D1288FC128AE32227
:068E9700128C74C20B22D4
:087DA200900988EDF0A3EBF05D
:107DAA00A3E004F090098DEFF0A3EBF0900988E0CE
:107DBA00FF90098DE0FED39F5068124FAD90098F56
:107DCA00F0A3EFF090098E124F59900991F0A3EFAA
:107DDA00F0E490098BF0A3F0900991124FEC90090E
:107DEA008F124F8F1280A7900990E004F0700690CE
:107DFA00098FE004F090098CE004F0700690098B7A
:107E0A00E004F0C390098CE0941890098BE0940187
:107E1A0040C6128AE390098DE004F0A3E004F00260
:107E2A007DB6900402E0FF900989E0D39F5009A330
:087E3A00E0C39F400312866EB5
:017E4200221D
:0F70CD009009AAEDF09009A9EFF09009ABEBF054
:1070DC009009B0EFF0A3EBF09009AAE0FF9009B093
:1070EC00E0D39F40030271C7A3124F59124F9E90D9
:1070FC0009B2E0FEA3E0FFC39418EE9401502A906D
:10710C0009AC124F92741B2FF58274053EF583ED7A
:10711C00F09009ADE004F070069009ACE004F012B8
:10712C004FF370CB124FFA80C6124F569009AEF047
:10713C00A3EFF09009B1124F59124F9E9009AC1267
:10714C004FEC9009AE124F8F1280A79009AFE0045C
:10715C00F070069009AEE004F0124FF37003124F7A
:10716C00FAC39009B3E094189009B2E0940140CCB2
:10717C00124F569009AE124FA19009B2E0FCA3E059
:10718C00FDC39418EC940150229009AE124FECAF51
:10719C00F0FE741B2DF58274053CF583E0FD128026
:1071AC00A7124FF370D3124FFA80CE128AE39009D4
:1071BC00B0E004F0A3E004F00270E4900402E0FFFD
:1071CC009009ABE0FED39F50209009A9E0FDA3E00D
:1071DC00C39DFDE49400FCEE7A002DFDEA3CFCC35B
:1071EC00ED9F7480F86C985013900402E0FF9009A6
:0F71FC00A9E0D39F5009A3E0C39F400312866E02
:01720B002260
:038017009009BE0F
:10801A00124FDB128E919009BFE0FE9009BEE090EC
:10802A0009C61250019009C2F09009C0E0FF9009F8
:10803A00C6E0FCA3E0FD7B017A05791B9009E012FA
:10804A004F87128B749009C7E02418F09009C6E094
:10805A003401F09009C2E0FF124FC9A374FFF0A3E4
:10806A00EAF0A3E9F0128E769009C3A3E0FAA3E03E
:10807A00AE02FF7A05791B124F821288FC128AE33C
:10808A009009C2E004F0E0C3941E409D900784E08A
:0C809A00FF128E1F9009C1E024FF92AF7E
:0180A60022B7
:038220009009D1F1
:10822300124FDB128E919009D2E0FE9009D1E090BB
:1082330009D61250019009D5F09009D5E0FFC394F7
:108243001E504175F018EF124F5EFE9009D8F0FAF8
:10825300A3EFF0FB9009D3E0FF9009D6E0FCA3E085
:10826300FDA9037BFF9009E8124F87128CC4900984
:10827300D7E02418F09009D6E03401F09009D5E056
:1082830004F080B5900784E0FF128E1F9009D4E0BC
:0482930024FF92AF83
:0182970022C4
:107B1C00E4900403F0A3E054F8F054F7F0E4900A76
:107B2C0066F0900A66E0FFC39433501B75F002EFC9
:107B3C00A42405F582E5F03404F583E4F0A3F09079
:107B4C000A66E004F080DB9004657408F0A3E4F0AE
:107B5C00900A66F0900A66E0FFC394104003027C22
:017B6C001CFC
:107B6D00EF75F00BA4246BF9740435F0FAA37401CE
:107B7D00F0A3EAF0A3E9F0124F72F9E4124F6FF996
:107B8D00900001E4124B6A900002E4F5F0124CA152
:107B9D00900004E4124B6A900005E4124B6AE9244C
:107BAD0006124FC254C0124F6F2407124FC254F821
:107BBD00124B5854C7124F6F2408124FC254F8126B
:107BCD004B5854F7124B5854EF124B5854DF124B7D
:107BDD005854BF124B58547F124F6F2409124FC285
:107BED0054FE124B5854F94402124B5854C74428B2
:107BFD00124F6F240A124FC254F84405124B5854B9
:067C0D00C74408124B58A9
:097C1300900A66E004F0027B60B7
:017C1C002245
:03000000024000BB
:03000300025003A5
:03000B000250069A
:030013000250098F
:03001B0002500C84
:0300230002500F79
:03002B000250126E
:0300330002501563
:03003B0002501858
:0300430002501B4D
:03004B0002501E42
:0300530002502137
:03005B000250242C
:0300630002502721
:03006B0002502A16
:0300730002502D0B
:03007B0002503000
:03008300025033F5
:03008B00025036EA
:03009300025039DF
:03009B0002503CD4
:0300A30002503FC9
:10400000787FE4F6D8FD9000007F007E20E4F0A3E6
:0A401000DFFCDEFA75813502405531
:10401A0002503CE493A3F8E493A34003F68001F230
:10402A0008DFF48029E493A3F85407240CC8C333A7
:10403A00C4540F4420C8834004F456800146F6DF76
:10404A00E4800B010204081020408090720CE47E88
:10405A00019360BCA3FF543F30E509541FFEE4936B
:10406A00A360010ECF54C025E060A840B8E493A332
:10407A00FAE493A3F8E493A3C8C582C8CAC583CA5D
:10408A00F0A3C8C582C8CAC583CADFE9DEE780BE15
:017347000045
:1049C700E709F608DFFA8046E709F208DFFA803ED2
:1049D70088828C83E709F0A3DFFA8032E309F608BF
:1049E700DFFA8078E309F208DFFA807088828C8327
:1049F700E309F0A3DFFA806489828A83E0A3F608DB
:104A0700DFFA805889828A83E0A3F208DFFA804CB4
:104A170080D280FA80C680D4806980F2803380108B
:104A270080A680EA809A80A880DA80E280CA8033F4
:104A370089828A83ECFAE493A3C8C582C8CCC5836C
:104A4700CCF0A3C8C582C8CCC583CCDFE9DEE7803C
:104A57000D89828A83E493A3F608DFF9ECFAA9F0BB
:104A6700EDFB2289828A83ECFAE0A3C8C582C8CC11
:104A7700C583CCF0A3C8C582C8CCC583CCDFEADE2A
:104A8700E880DB89828A83E493A3F208DFF980CC8C
:104A970088F0EF60010E4E60C388F0ED2402B40485
:104AA7000050B9F582EB2402B4040050AF2323452C
:064AB7008223904A1773F0
:104ABD00C2D530F707B2D563F0FF05F030E70CB281
:104ACD00D5F4048463F0FF05F080018430D502F441
:024ADD000422B1
:104ADF00BB010689828A83E0225002E722BBFE02D5
:094AEF00E32289828A83E4932208
:104AF800BB010CE58229F582E5833AF583E0225073
:104B080006E92582F8E622BBFE06E92582F8E222BC
:0D4B1800E58229F582E5833AF583E49322D6
:104B2500BB010FF8E58229F582E5833AF583E02894
:104B3500F0225009C58229F8E58226F622BBFE0936
:104B4500C58229F8E22582F222F8EA2583F583E970
:034B550093282280
:104B5800BB010689828A83F0225002F722BBFE013C
:024B6800F32236
:104B6A00F8BB010DE58229F582E5833AF583E8F081
:104B7A00225006E92582C8F622BBFE05E92582C82D
:024B8A00F22215
:104B8C00EF8DF0A4A8F0CF8CF0A428CE8DF0A42E3D
:024B9C00FE22F7
:104B9E00BC000BBE0029EF8DF084FFADF022E4CCFB
:104BAE00F875F008EF2FFFEE33FEEC33FCEE9DECC4
:104BBE00984005FCEE9DFE0FD5F0E9E4CEFD22ED0A
:104BCE00F8F5F0EE8420D21CFEADF075F008EF2F54
:104BDE00FFED33FD4007985006D5F0F222C398FD45
:054BEE000FD5F0EA22E2
:104BF300C5F0F8A3E028F0C5F0F8E582158270024D
:064C03001583E038F022E9
:104C0900A3F8E0C5F025F0F0E5821582700215835E
:064C1900E0C838F0E822BB
:104C1F00BB010A89828A83E0F5F0A3E02250068760
:104C2F00F009E71922BBFE07E3F5F009E319228922
:0B4C3F00828A83E493F5F07401932255
:104C4A00BB0110E58229F582E5833AF583E0F5F0A8
:104C5A00A3E0225009E92582F886F008E622BBFE85
:104C6A000AE92582F8E2F5F008E222E5832AF583CB
:084C7A00E993F5F0A3E9932290
:104C8200BB010A89828A83F0E5F0A3F0225006F77D
:0F4C920009A7F01922BBFE06F3E5F009F319227A
:104CA100F8BB0111E58229F582E5833AF583E8F045
:104CB100E5F0A3F0225009E92582C8F608A6F02202
:0D4CC100BBFE09E92582C8F2E5F008F222E9
:104CCE00E88FF0A4CC8BF0A42CFCE98EF0A42CFC85
:104CDE008AF0EDA42CFCEA8EF0A4CDA8F08BF0A403
:104CEE002DCC3825F0FDE98FF0A42CCD35F0FCEB62
:104CFE008EF0A4FEA9F0EB8FF0A4CFC5F02ECD3927
:0F4D0E00FEE43CFCEAA42DCE35F0FDE43CFC2293
:104D1D0075F008758200EF2FFFEE33FECD33CDCC4D
:104D2D0033CCC58233C5829BED9AEC99E5829840D0
:104D3D000CF582EE9BFEED9AFDEC99FC0FD5F0D6AD
:104D4D00E4CEFBE4CDFAE4CCF9A88222B800C1B9D7
:104D5D000059BA002DEC8BF084CFCECDFCE5F0CB15
:104D6D00F97818EF2FFFEE33FEED33FDEC33FCEB4E
:104D7D0033FB10D703994004EB99FB0FD8E5E4F909
:104D8D00FA227818EF2FFFEE33FEED33FDEC33FCF6
:104D9D00C933C910D7059BE99A4007EC9BFCE99AEA
:104DAD00F90FD8E0E4C9FAE4CCFB2275F010EF2F2F
:104DBD00FFEE33FEED33FDCC33CCC833C810D7072F
:104DCD009BEC9AE899400AED9BFDEC9AFCE899F86A
:0E4DDD000FD5F0DAE4CDFBE4CCFAE4C8F922FD
:10883500C2D5E830E70FB2D5E4C39BFBE49AFAE46E
:1088450099F9E498F8EC30E717B2D512886B124D18
:1088550059E4C39BFBE49AFAE499F9E498F8800398
:10886500124D5930D50DE4C39FFFE49EFEE49DFDF6
:04887500E49CFC2261
:0D4DEB00CFF4CFCEF4CECDF4CDCCF4CC225D
:104DF800EB9FF5F0EA9E42F0E99D42F0EC6480C832
:064E080064809845F022D1
:104E0E00EB9FF5F0EA9E42F0E99D42F0E89C45F0FA
:014E1E002271
:104E1F00E8600FECC313FCED13FDEE13FEEF13FF71
:034E2F00D8F12295
:104E3200E86010ECA2E713FCED13FDEE13FEEF1396
:044E4200FFD8F02283
:104E4600E8600FEFC333FFEE33FEED33FDEC33FCCA
:034E5600D8F1226E
:104E59007401FF3395E0FEFDFCA3A3A3E0CF2FF07F
:104E6900E582158270021583E0CE3EF0E582158257
:104E790070021583E0CD3DF0E5821582700215833D
:054E8900E0CC3CF0222A
:0C4E8E00ECF0A3EDF0A3EEF0A3EFF02297
:104E9A00A8828583F0D083D082124EB1124EB1120D
:104EAA004EB1124EB1E473E493A3C583C5F0C58332
:104EBA00C8C582C8F0A3C583C5F0C583C8C582C862
:014ECA0022C5
:0C4ECB00A42582F582E5F03583F58322F2
:104ED700D083D082F8E4937012740193700DA3A36A
:104EE70093F8740193F5828883E47374029368607E
:064EF700EFA3A3A380DF7E
:104EFD00EC8EF0A4CCC5F0CCCDF8EFA4CEC5F02D42
:104F0D00FDE43CFCE8A42EC8C5F03DFDE43CFCEFFF
:0D4F1D00A4FFE5F028FEE43DFDE43CFC228D
:104F2A00EF4E6012EF60010EEDBB010B89828A839E
:104F3A00F0A3DFFCDEFA2289F05007F709DFFCA9AB
:0C4F4A00F022BBFEFCF309DFFCA9F02202
:00000001FF
